:1000000055AA55AA0200000036700000000000004A
:1000100065F2000000000000FD100000000000007C
:100020000000000000000000FD10000080610000E2
:1000300000080000000000000000000043A982103A
:10004000C03125F45F1800003FCEDA0BA0E7FFFFB8
:1000500000021000E1000000A34D0000A10100001B
:10006000ED010000390200008502000000000000E0
:10007000000000000000000000000000AB4D000088
:10008000B34D000000000000D1020000BB4D000095
:10009000C34D0000CF4D0000D74D0000E34D0000E0
:1000A000EF4D0000FB4D0000034E00000F4E00001E
:1000B0005B4E0000DF0200001B4E0000234E0000DC
:1000C00000000000334E00005D4E00005F4E000057
:1000D0006B4E00006D4E00006F4E00004B4E000056
:1000E000534E00003B4E0000434E0000714E000096
:1000F000734E00007F4E00002B4E000000000000F9
:1001000000000000000000000000000000000000EF
:1001100065F2000001000140000000000000000046
:1001200000000000000000000000000000000000CF
:1001300000F002F800F03AF80AA090E8000C8244BF
:100140008344AAF10107DA4501D100F02FF8AFF29C
:10015000090EBAE80F0013F0010F18BFFB1A43F0A5
:1001600001031847105E0000405E0000103A24BFF3
:1001700078C878C1FAD8520724BF30C830C144BF0C
:1001800004680C607047000000230024002500264E
:10019000103A28BF78C1FBD8520728BF30C148BFEA
:1001A0000B6070471FB51FBD10B510BDDFF80CD038
:1001B000FFF7F8FF04F01FFF05F038FB0002100006
:1001C00003B4FFF7F1FF03BC05F03AFB40BA7047F8
:1001D000C0BA704772B6784600F10A004DF8080CB4
:1001E00062B630BF00BF704740BA7047C0BA7047B0
:1001F00011484FF00F0100F8011B4FF0010100F80A
:10020000011B4FF0020100F8011B4FF0000100F844
:10021000011B00F8011B00F8011B00F8011B00F88E
:10022000011B1EF0040F0CBFEFF30880EFF30980F1
:100230004FF0020103F054BD0002002011484FF0BE
:100240000F0100F8011B4FF0010100F8011B4FF0F6
:10025000030100F8011B4FF0000100F8011B00F83A
:10026000011B00F8011B00F8011B00F8011B1EF028
:10027000040F0CBFEFF30880EFF309804FF0030188
:1002800003F02EBD0002002011484FF00F0100F8CE
:10029000011B4FF0010100F8011B4FF0040100F8B1
:1002A000011B4FF0000100F8011B00F8011B00F8D2
:1002B000011B00F8011B00F8011B1EF0040F0CBF0E
:1002C000EFF30880EFF309804FF0040103F008BD5D
:1002D0000002002011484FF00F0100F8011B4FF001
:1002E000010100F8011B4FF0050100F8011B4FF060
:1002F000000100F8011B00F8011B00F8011B00F8C9
:10030000011B00F8011B1EF0040F0CBFEFF3088067
:10031000EFF309804FF0050103F0E2BC000200207A
:1003200000B504F05DFD5DF804EB00F02FB81EF0A1
:10033000040F0CBFEFF30880EFF309804FF00001CA
:1003400003F0CEBC0A484FF0FF0101704FF00000EF
:1003500080F311884FF0000080F3098805484FF0C2
:100360000201017062B604484FF08051016070478D
:1003700022ED00E00703100004ED00E002484FF01A
:10038000805101607047000004ED00E04FF0200054
:1003900080F31188EFF3098098B112480068124980
:1003A0000968884217D0EFF309800E49096820E9EF
:1003B000F00F886000B50B48006804F0F0FE5DF8AF
:1003C00004EB084808490A68026000688168B1E8DF
:1003D000F00F81F309884EF0040E4FF0000080F317
:1003E00011887047080310000C031000EFF3118010
:1003F0004FF0200181F31188704700004FF000009A
:1004000080F311887047000062B6704772B670477B
:1004100010B5022000F00AFA032000F007FA0420C9
:1004200000F004FA052000F001FA062000F0FEF9C1
:10043000072000F0FBF9082000F0F8F9092000F08F
:10044000F5F90F2000F0F2F94FF00051002001F80B
:100450004A0F8871F022CA710F224A70F949086266
:1004600088620863886008618861C8604861C86103
:100470004862C86248630621022000F0F6F90621AE
:10048000032000F0F2F90621042000F0EEF9062125
:10049000052000F0EAF90621084600F0E6F90621F9
:1004A000072000F0E2F90621082000F0DEF904211F
:1004B000092000F0DAF906210F2000F0D6F9022019
:1004C00000F0C8F9032000F0C5F9042000F0C2F9DB
:1004D000052000F0BFF9062000F0BCF9072000F06D
:1004E000B9F9082000F0B6F9092000F0B3F90220AC
:1004F00000F091F9032000F08EF9042000F08BF950
:10050000052000F088F9062000F085F9072000F0AA
:1005100082F9082000F07FF9BDE81040092000F0C2
:100520007AB94FF00051C98C4FEA90100A06C549BC
:1005300001D5C54A00E0C54AB2FBF0F0086070473B
:100540004FF0005090F84A00000700D0012070479B
:100550007047BF4900200860BA498860C86070478A
:10056000B84AD160642148430A2190FBF1F0B0F50C
:10057000803F06DBA0F57F40FF3890604FF6FF70AC
:1005800002E0002180B2916000F07FB9AD4910B562
:100590008868B0F5803F06DBA0F57F40FF388860B3
:1005A0004FF6FF7003E030B10022C0B28A60BDE8B0
:1005B000104000F06AB9CA68FFF7CBFF12B1BDE87E
:1005C000104010470020FFF7C3FF10BDA0490020D6
:1005D000091D08609B49086148617047994A51614B
:1005E000642148430A2190FBF1F0B0F5803F06DB1F
:1005F000A0F57F40FF3810614FF6FF7002E0002148
:1006000080B2116100F04BB98E4910B50869B0F5A0
:10061000803F06DBA0F57F40FF3808614FF6FF7092
:1006200004E0002806DD002280B20A61BDE8104027
:1006300000F035B94A69FFF7C9FF12B1BDE81040B3
:1006400010470120FFF784FF10BD814900200831C9
:1006500008607C498861C86170477A4910B588692B
:10066000B0F5803F06DBA0F57F40FF3888614FF68C
:10067000FF7003E030B1002280B28A61BDE8104013
:1006800000F017B9CA69FFF7E0FF12B1BDE81040EA
:1006900010470220FFF75CFF10BD6D4900201031AC
:1006A00008606849086248627047664910B5086A80
:1006B000B0F5803F06D3A0F57F40FF3808624FF6C3
:1006C000FF7003E030B1002280B20A62BDE8104042
:1006D00000F0F9B84A6AFFF7E0FF12B1BDE8104038
:1006E00010470420FFF734FF10BD59490020143192
:1006F000086054498862C8627047524AD1621168E2
:1007000048430A21B0FBF1F0B0F5803F06DBA0F5CD
:100710007F40FF3890624FF6FF7002E0002180B208
:10072000916200F0DBB84FF00050B0F85A00454934
:10073000096908447047434910B5886AB0F5803F9D
:1007400006D3A0F57F40FF3888624FF6FF7003E0C4
:1007500030B1002280B28A62BDE8104000F0BEB81D
:10076000CA6AFFF7C2FF12B1BDE81040104705206A
:10077000FFF7EEFE10BD4020C10581F82100704753
:10078000334800211C3001604FF000524FF6FF71DA
:10079000A2F866100121016070472D4900201C312C
:1007A000086070474FF0005090F82110C90606D538
:1007B00010F8211F21F01001017001207047002066
:1007C000704710B504460F2000F044F80F2000F0E9
:1007D00022F81C4844604FF00050C18C090602D535
:1007E0004EF6602101E04AF6C871416518490120C2
:1007F000B8310860091D086010BD10B50F2000F069
:1008000015F84FF00050C06C0E4920F07F40496849
:10081000BDE81040084700F01F0201219140400947
:10082000800000F1E020C0F80011704700F01F02C6
:10083000012191404009800000F1E020C0F88011C2
:100840007047000000021000C0270900D0DD06003C
:100850004009002200F01F02012191404009800060
:1008600000F1E020C0F88012EAE74907090E0028ED
:1008700006DA00F00F0000F1E02080F8141DDFE739
:1008800000F1E02080F80014DAE71A4900220A603B
:100890004FF00052A2F8580001200860D0E7154937
:1008A0000022091D0A60CA06A2F85A000120086049
:1008B000C6E71049002208310A608A06A2F85C00E7
:1008C00001200860BCE70B49002210310A604FF09C
:1008D0000052A2F8600001200860B1E7054900223B
:1008E00014310A604FF00052A2F862000120086043
:1008F000A6E700004009002210B55B4C00202060F4
:100900005A4800F09BFD0120206010BD10B54FF04B
:10091000E0214FF08060C1F88001C1F880025449A5
:10092000A02081F80004FFF7E7FF4FF00051C88CCA
:10093000CA8C00F00300120600EB400001D54D4ABE
:1009400001E04C4A303A12F8203001F8983F02EBAF
:10095000800042784A7082788A70C278CA700279C0
:100960000A7142794A7182798A71C279CA71027AAE
:100970000A72427A4A72827A8A72C07AC87210BD4A
:1009800070B54FF0005400F07F00049D84F88D0096
:1009900084F88E10A4F8942001213748002283B1F6
:1009A000C0F8801194F8913023F0700384F89130EE
:1009B00094F89130702606EA05152B4384F891309F
:1009C00001E0C0F8802114F8923F23F03403237033
:1009D000C0F84422C0F84012D0F89C110129FBD184
:1009E00070BDF0B54FF00054DDE90765DDE905C7DE
:1009F00000F07F0084F88D0084F88E10A4F8942015
:100A000084F88F30A4F896C001211B48002287B1DA
:100A1000C0F8801194F8913023F0700384F891307D
:100A200094F89130702707EA05152B4384F891302C
:100A300001E0C0F8802114F8923F23F034032370C2
:100A4000237843F02003237016B1C0F8481201E068
:100A5000C0F84822C0F84422C0F84012D0F89C11D7
:100A60000129FBD1F0BD000084140022AA820600F7
:100A70001AE000E0885800000010002237480121E9
:100A800001600021016070473548012101600021AB
:100A90000160704700B54FF0E0230122C3F88021C8
:100AA00003F5C073FFF7F0FFFFF7E8FF2C480838A5
:100AB0000260A02083F88002C3F8002143F8802C54
:100AC00000BD2749083910B1002008607047012097
:100AD000FBE723480121783801600021016070475D
:100AE00010B572B61F490C78002104E01D4A521C53
:100AF000525C4254491CA142F8DB40F6FC0000F075
:100B00009DFC62B6204610BD144901201C390860C6
:100B10007047144820300078124921310978401A72
:100B200000F03F0070474FF00051027881F800223A
:100B3000427881F80122827881F80222C27881F815
:100B40000322027981F80422427981F80522827910
:100B500081F80622C07981F8070270475C84002280
:100B6000940500220004002010B50A2000F05AF875
:100B70000B2000F057F80A2000F05FF80B2000F07F
:100B80005CF805210A2000F063F805210B2000F035
:100B90005FF84FF000507F2100F8351F4170C170A1
:100BA0000021C17101724172817210BD0123834025
:100BB000D8B24FF00053002993F8361001D001430A
:100BC00000E0814383F8361013F8381F0AB101435F
:100BD00000E081431970704701238340D8B24FF081
:100BE0000053002993F83C1006D0014383F83C10D1
:100BF00093F83E10014305E0814383F83C1093F8DD
:100C00003E10814383F83E1013F83D1F22B101438B
:100C100019709978014303E08143197099788143F1
:100C20009970704700F01F02012191404009800037
:100C300000F1E020C0F88011704700F01F02012190
:100C400091404009800000F1E020C0F88012704718
:100C50004907090E002806DA00F00F0000F1E02035
:100C600080F8141D704700F1E02080F800147047F0
:100C70007047FE4BFE4A998A814203D2401AD080C7
:100C8000084601E00021D180DA68FA491047F748A8
:100C900010B500698047F649C88810B1BDE810401A
:100CA000E7E78968002903D0BDE810400120084724
:100CB00010BDEE4810B500698047ED4C4FF00000C4
:100CC000A16819B188470020A06010BDFFF7D0FFD0
:100CD00010BDE749CA780B7952005A43E34B0878B4
:100CE000D2B29B6840F48070C96818470146182248
:100CF000DE4804F0A1BC38B5DD4A817913231171B7
:100D00004179D170027901F0070102F01F028DF8DC
:100D100000208DF80110C078032200F01F008DF82C
:100D20000200D248694644681846A04738BDF8B565
:100D30000446007CCD4DC0F34002014662F35F01E2
:100D4000C0F3800241EA8201C0F3C00241EAC2015D
:100D5000C0F3001241EA0211C0F3401241EA42110D
:100D60008DF800108109607C272300F0010241EA20
:100D70000211C0F3400041EA40108DF80100607C90
:100D8000C0F38001C0F3C00241EA0211C0F30012B7
:100D900041EA4211C0F3401241EA8211800941EA5E
:100DA000C0108DF802006E68032269461846B047ED
:100DB000E0792B23C0F38002014662F39F01C0F368
:100DC000C10241EA0211C0F3401041EA80108DF8DF
:100DD0000000607CA17CC00901F0030140EA011021
:100DE0008DF801006E68022269461846B0472D262C
:100DF0002B680122694630469847A17C9DF8000087
:100E0000C1F3800108438DF800006B680122694638
:100E100030469847F8BD10B50446FFF76CFF2046F2
:100E200000F04FF92046BDE8104080E738B53D217D
:100E30008DF800108D49044612204B680122694646
:100E40009847A088FFF715FF38BD10B5044600F09D
:100E50007AF92046BDE81040E8E7F8B5834C122542
:100E60000646236801226946284698479DF80000F7
:100E7000012240F008008DF80000636869462846AA
:100E800098474825236801226946284698479DF8D7
:100E90000000012220F0060040EA46008DF8000024
:100EA00063686946284698472368012269462846B0
:100EB00098479DF80000012240F001008DF80000E5
:100EC0006368694628469847F8BD38B5674D482499
:100ED00001222B686946204698479DF800000122B0
:100EE00020F001008DF800006B68694620469847A5
:100EF00038BD38B55D4D2A2401222B68694620464D
:100F000098479DF80000012220F0100040F00100F9
:100F10008DF800006B6869462046984738BD38B5A3
:100F2000524D2A2401222B686946204698479DF895
:100F30000000012220F001008DF800006B68694676
:100F40002046984738BDF8B5484C442506462368E6
:100F500001226946284698479DF80000012240F08A
:100F600082008DF8000063686946284698472D2561
:100F7000236801226946284698479DF8000001220F
:100F800020F0FC0040F08E008DF800006368694698
:100F90002846984714252368012269462846984721
:100FA0009DF80000012220F0070040F001008DF8BC
:100FB0000000636869462846984715252368012282
:100FC0006946284698479DF8000006F01F0120F06A
:100FD0001F0001438DF8001063680122694628460E
:100FE0009847F8BD2DE9F843204C1325174688464D
:100FF00081462368012269462846984701269DF8C4
:10100000000006FA08F120F01F0001F01F01014363
:101010008DF80010636832466946284698472725B0
:10102000236801226946284698479DF80000BE4083
:1010300020F03F0006F03F0101438DF80010636887
:1010400001226946284698472E25236801226946D1
:10105000284698479DF80000012240F00C008DF8CA
:101060000000636869462846984705E018031000A9
:10107000380210003F0C00003E2023680122694620
:1010800098479DF8000000F0300189F80010BDE895
:10109000F883554B40F480701B681847524B40F45E
:1010A00080705B68184701B506209DF8001001228A
:1010B00001F01F018DF800104B494B6869469847B5
:1010C00008BDFEB5494D0446007828706078687008
:1010D000454EA078A870312733680122694638460A
:1010E0009847E07940069DF8000002D540F02000C6
:1010F00001E020F020008DF80000E179090602D51A
:1011000040F0800001E020F080008DF8000073685E
:10111000012269463846984721893220C1F30801E7
:10112000ADF80010E168CDF8021029788DF80610AE
:1011300069788DF80710A9788DF80810736809226E
:1011400069469847FEBD70B504460168274886B0D9
:10115000254D8160A168C160E1680161217C162094
:1011600001F001018DF80010617C8DF80110A17C67
:101170008DF8021000218DF80310A18A0F22C1F30F
:101180000C01ADF80410E18AC1F30B01ADF80610B3
:10119000218BC1F30B01ADF80810618BC1F30B017A
:1011A000ADF80A10A18BC1F30B01ADF80C10A17FB3
:1011B0008DF80E106B686946984731262B6801221E
:1011C00004A9304698479DF81000E17F20F01F00E9
:1011D00001F01F0101438DF810106B68012204A972
:1011E0003046984706B070BD180310003802100052
:1011F0004FF0E0214FF48030C1F88001C1F8800247
:101200007249A02081F80004704730B5704C012568
:101210002560E50603F03F0385F86B30002304E00A
:1012200051F8235040F823505B1C9342F8DB002018
:10123000206030BD30B595B00446302104F058FA36
:101240006448006800906348001D00680190614890
:101250000830006802905F480C30006803905D48D9
:101260001030006804905B481430006805905948BD
:1012700018300068069057481C30006807905548A1
:101280002030006808905348243000680990514885
:10129000283000680A904F482C3000680B904D4869
:1012A000303000680C904B48343000680D9049484D
:1012B000383000680E9047483C3000680F90454831
:1012C0004030006810904348443000681190414815
:1012D0004830006812903F483F494C306FF002059B
:1012E00000681390009888424DD1A810A061206139
:1012F0002060A062E062E061206203A8029900F031
:101300006FF8019981423ED10B9845F2AA5180B203
:10131000884208D10498C0B2A061139A92B28A425E
:1013200000D0801DE0610C9880B2884217D10398EC
:10133000039A00F47F40D2B240EA0240039AC2F31B
:1013400007421043254A904203D30598C0F3012079
:1013500000E000202061059800F00F0020600D984B
:1013600080B2884201D10698A0620E9880B288426D
:1013700001D10798E0620F9880B2884201D10898A5
:10138000206215B030BDA56125612560A562E562CA
:10139000E5612562F5E710B50446142104F0A8F9CB
:1013A0000C487C38006820600A488038006860601B
:1013B000084878380068A060064874380068E06023
:1013C000044870380068206110BD000010E000E0A3
:1013D000441B0022B41E04005C000D6000010200EA
:1013E000F0B5074600200346184E10E057F823508A
:1013F00003224FEAC20C45FA0CF484EA2064E4B2FA
:10140000521E56F8244084EA0020F2D55B1C8B4221
:10141000ECDBF0BD70B5054600200C4C0246103CDC
:1014200009E0AB5C521C03F00F0604EB1313A65D3E
:101430001B78304418448A42F3DB70BD08B5009035
:10144000401E00900028FBDC08BD0000C8580000CA
:101450004FF00051C88C4C4A00F0030012687AB17A
:1014600001280AD0022806D0032802D04FF41670B3
:101470000EE046200CE096200AE04FF4967007E05C
:1014800001280ED002280AD0032806D04FF4E170BC
:10149000401E21F8520F088070473220F8E76E2076
:1014A000F6E7DC20F4E748F61971480720F82A1F10
:1014B0000B2180F83E1000214183022180F8C010EA
:1014C0004FF008510120C1F8D4032F499839086022
:1014D0002E49086070474FF0005141F29840C8848F
:1014E000B6E74FF0005140F29A70C884B0E74FF071
:1014F0000050C08CA0F5A051983901D00020704751
:10150000012070474FF000518A8C60F304028A84F6
:1015100070471F48016841F00401016070471C4892
:10152000016821F00401016070474FF0005108810B
:101530007047174928310968016015491831096851
:10154000416013491C3109688160114920310968E3
:10155000C1600F492C31096801610D490C390968D6
:1015600041610B4914310968816170474FF00050A7
:10157000808870474FF00050807970474FF00051DD
:101580004C2081F820007047DC040022EC1B002274
:1015900010ED00E030B41DC8484981E81D0001216C
:1015A00030BC002003F02CBE2DE9F84F4448012444
:1015B000006810F86C5F417890F846004D4300F0E9
:1015C000030004FA00FA3D486421103004F090F85A
:1015D0003C4803F0BFF93B483B490471097809B91D
:1015E00002210171DFF8D480002408F1100B36E0ED
:1015F000DFF8D090032735490026C9F80010484687
:1016000003F0ACF900226B460121104603F048FEBE
:101610000121002003F023FE98F8000060B102F0E1
:1016200092FB7F1E002F0AD0E9DC76B34FF000005A
:101630005946D8F804200FE04FF00106F5E74FF0C7
:10164000040003F080F9F0E751F8203032F910700F
:101650003B4441F82030401CA842F5DB641C544553
:10166000C6DB012E11D1164900205C46184A0B68D2
:1016700009E093F8B26054F8201006F003063141F7
:1016800022F81010401CA842F3DB12490120087018
:10169000BDE8F88F10B50446002003F062FE02207A
:1016A00003F05FFEE00701D0FFF77EFF022003F0AA
:1016B00073FEBDE81040002003F06EBE3003100042
:1016C000E00210004C021000050310004515000058
:1016D000523C01208C02100010B51C4C40F2FF114E
:1016E0002068FFF77DFE2168C1F8FC07FFF748F886
:1016F00000213F200EF1ACFAFFF742F82168BDE867
:1017000010403F234FF400721148FFF77EBD10B523
:1017100040F2FF310F48FFF763FE0E49C1F8FC0F9E
:10172000FFF72EF800213D200EF192FA00213E2015
:101730000EF18EFAFFF724F8BDE810403D234FF478
:10174000806204490448FFF760BD0000E002100019
:10175000F0EF03004C000120F0CF030030B41DC8AF
:101760004F4981E81D00012130BC002003F048BD35
:1017700010B5002003F0F5FDFFF7BBFB00F064F8A7
:101780000446FFF7CCFB012C04D13C224549A020A4
:10179000FFF77FFC002003F0FFFD012010BD10B516
:1017A000FEF714FFBDE81040822002F0DFBA2DE9F9
:1017B000F047002003F0D5FD00253B4F4FF0360ADF
:1017C0006E1EA846E8B2FFF76EFC0020FFF745FB4F
:1017D0003C683868A042FCD03868A042FCD133494C
:1017E0006420FEF7FBFEFEF79EFF81463868A042AC
:1017F000FCD03868A042FCD1FEF795FF0446FFF705
:1018000064FBFEF7E3FEA9EB040080B2B0EB0A0034
:1018100001D4014600E04142B14204D2002800DA7E
:1018200040420646A8466D1C6DB2202DCADB1D49FC
:1018300008F0FF00743981F8B000FFF734FCBDE810
:10184000F047002003F0A8BDFEB50025684603F070
:1018500081F8174800900320114E8DF804000446CB
:10186000684603F07BF8002202AB0121104603F02A
:1018700017FD0121002003F0F2FC307838B1641E1E
:1018800002F061FA002C05D0EADC2846FEBD4FF0DC
:101890000105FAE74FF0020003F055F8F5E7000004
:1018A000A4031000C0000120981B00224F17000065
:1018B0000D17000030B41DC88E4981E81D000121BC
:1018C00030BC002003F09CBC2DE9F84F8A4800682A
:1018D00010F86C4F40784443FEF75FFF8548642161
:1018E000103003F005FF3221844803F0DFFE32217F
:1018F000834803F0DBFE814842F21071323003F07E
:10190000D5FEDFF8F8A10020AAF1320A47F6FF71F0
:10191000AAF1320BCA4304E02AF810102BF8102069
:10192000401CA042F8DB774803F014F87549012009
:1019300000250871DFF8CC9103267349DFF8B481E4
:101940000027C9F80010484603F008F800226B464B
:101950000121104603F0A4FC0121002003F07FFCCC
:1019600098F80000C0B102F0EEF9761E002E16D0F5
:10197000E9DCBFB36148D8F8041005FB04F200F1BC
:101980003200DFF8708100EB42034FF00000564652
:101990005F4608F1100823E04FF00107E9E74FF038
:1019A000040002F0D0FFE4E731F8102023F8102003
:1019B00058F8202031F910C0624448F8202031F94D
:1019C000102037F910C0624501DD27F8102031F9E9
:1019D000102036F910C0624501DA26F81020401CAC
:1019E000A042E1DB6D1CC82DA4DBDFF808810020DC
:1019F000C821424D52465B4608F110080EE033F90B
:101A0000106032F91070F61B761025F8106058F847
:101A1000206096FBF1F648F82060401CA042EEDB07
:101A2000364F0020364E3237894615E0002258F8EE
:101A30002030114601FB040C37F91CC0BCEB030C31
:101A400001D5CCF1000C491C6244C829F2DB92FBA1
:101A5000F9F126F81010401CA042E7DB002707E050
:101A600036F9172035F91710F8B202F067FB7F1C22
:101A7000A742F5DBBDE8F84FFEF782BE2DE9F8433B
:101A800000248DF80040FEF788FE002003F069FC7A
:101A9000194D286890F86B00FFF755FA2F6800255C
:101AA000A1464FF00108A1370024785D08FA04F63A
:101AB0008DF8009006400DD0224629466846FFF773
:101AC00091FA9DF80000202804D1324629460520CD
:101AD00002F031FA641CE4B2062CE6D36D1CEDB2C0
:101AE000052DE1D3002003F057FCFEF749FEBDE8C9
:101AF000F8830000B4031000E0021000B0100120D1
:101B0000F2370120540210006518000010B5044699
:101B10000221002003F074FB0F48046010BD08B5DB
:101B20000E48FEF74EFE00226B460221104603F0DF
:101B3000B7FB0221002003F092FB094855220168FF
:101B400005480A7100684871020A8A71020CCA715C
:101B5000FEF7E7FC08BD00005C021000BD1A0000A3
:101B6000E402100008B50024DFF85881564F4FF406
:101B70000049264600226B464146104603F090FB82
:101B80000098800319D5FEF741FC504804680660B0
:101B9000FEF73AFCE00701D0FFF709FEA00701D5E8
:101BA000FFF7E6FD00231A460121022002F0ADFAFC
:101BB0004FF40031002003F052FB0098000411D5CF
:101BC00000256D1CEDB2FFF7D3FD01286ED0032D6B
:101BD000F7D900224946082002F0ADF94946002015
:101BE00003F03DFB0098000510D5394804680660F5
:101BF0002046FFF74FFD4FF40061002003F02FFB5C
:101C00000023E1B21A46062002F07FFA0098C004D1
:101C10000CD5FFF784FF002301221946022002F0B1
:101C200074FA4FF48051002003F019FB00988004EF
:101C300006D5FFF751FD4FF40051002003F00FFBD4
:101C40000098400406D5FFF762FD4FF48041002064
:101C500003F005FB0098400311D5386890F8A00008
:101C6000C0070CD0FFF70AFF4FF48021002003F0DB
:101C7000F6FA00231A4619460C2002F046FA00989C
:101C800000037FF577AF386890F8A0008007F8D59B
:101C9000FFF71AFE4FF40021002003F0E0FA0023C2
:101CA0001A4619460E2002F030FA63E70120FFF7CA
:101CB000F1FCE1B20023C4F30722082002F025FA68
:101CC0008CE7000003F80F00E00210000003100092
:101CD000FC02100010B58143C80711D064480168A8
:101CE00041F0010101604FF40061002003F088FA27
:101CF00001220023BDE810401146052002F005BA7C
:101D000010BDFEF7F2BC10B5FEF7EFFC0121BDE8F7
:101D10001040084603F074BA5649012805D002283D
:101D200005D0032805D1042002E0022000E00320B2
:101D30000870704738B5002003F013FB4E48006868
:101D400010B1FFF7E9FF01E000F0CCF949484B4939
:101D50000078022813D003280ED0042812D00124C2
:101D60000025FEF7D6FE00B101256946032003F0E9
:101D700086FA009858B909E00868847AF0E708689C
:101D8000447AEDE70868B0F80B40E9E715B1142C88
:101D900000D2142420463A49FEF7AFFC0324394D03
:101DA00000F022FA012807D1287858B1641E01F00A
:101DB000CAFF002C0DD0F3DCBDE838404FF0000026
:101DC00003F0EABA304801683048006800F01CF9B6
:101DD000F2E7032002F0B7FDEEE770B52C48046887
:101DE0002C490D680C6095EA040F27D0214E2DB1C7
:101DF000A4B121462846BDE870406BE70220307050
:101E00001E4800680079000701D404203070214684
:101E10002846FFF75FFFBDE870408BE7FEF765FCE3
:101E20000121084603F01BFA0120307021462846A4
:101E3000FFF750FFBDE8704000F0F7B870BD10B577
:101E4000FEF753FC0121084603F009FA0949042072
:101E5000087000F0B1F8BDE810406BE710B5FEF770
:101E600044FC0121084603F0FAF9BDE8104061E79F
:101E7000FC02100070021000F4021000E0021000DA
:101E8000B71C0000280410007C021000780210002B
:101E9000EC021000740210002DE9FC5F0E460028D1
:101EA0001BD055490978042917D1002A15D1DFF82C
:101EB0004C91DFF84C81534DD9F800109246097AC5
:101EC00049070ED5A978491CC9B2A970032906D8BB
:101ED000018808EB460020F8021CBDE8FC9F85F84D
:101EE00002A0032003F03DFA454801906C78B5F953
:101EF00004B02878274640B941480F235A46009439
:101F0000801D019902F06EFB002734B93C4A5B4604
:101F1000921D901D019902F056FB39496F700C31EA
:101F2000B5F90420B5F90630002007E031F910407A
:101F30009C4201DD012404E0401CC0B29042F5DB6C
:101F40000024032003F028FAD9F8000090F8E307F2
:101F5000DA2823D1D8F80010C8F81210B8F8041005
:101F6000A8F81610D8F80610C8F81810B8F80A1013
:101F7000A8F81C10D8F80C10C8F81E10B8F81010EB
:101F8000A8F822101E48C8F824A0C8F828A01230CB
:101F9000A8F82CA04682A9788182C4822C70002CDB
:101FA0009BD0FFF7AEFEBDE8FC5F0121084603F0C1
:101FB00027B9144800787047124A012050700F4822
:101FC0000068017A4B0790F8711002D590F86C30D8
:101FD00001E090F8703059439180B0F84B00D08008
:101FE0000021074811709170C1600182C0F806108D
:101FF000418100F0A9BADFE770021000E002100092
:10200000243801206002100070B5054630480C46A7
:10201000224690F90D102F484068FFF73DFF2146FA
:102020002846BDE8704000F014B810B5032003F056
:1020300098F94821284803F05BFB274901200870E4
:10204000032003F0A9F90121BDE81040022003F0AC
:10205000D7B82DE9F041DFF884800746002698F8CC
:1020600000000D4604282CD047EA0504032003F0A5
:1020700078F9194A174B978115619868506098F85C
:10208000000004281FD0FF2111751070E0070DD04B
:102090001348016811F86C0F49784843906042007A
:1020A0000D485968163003F082FA0126032003F028
:1020B00073F9002E09D0BDE8F0410121022003F0A0
:1020C0009FB80C46D2E7197BDEE7BDE8F08100003F
:1020D00018051000280410005C05100070021000A4
:1020E000E00210002DE9F0417A4C0026DFF8E8818B
:1020F00020780227794D04280ED000F025FD012814
:1021000019D07748237802680320022B517B10D125
:1021100098F8003093B113E0FFF74BFF012803D08C
:1021200098F80000012804D16E49277001202E6024
:102130000870BDE8F08127702E60FAE7917B0420DB
:10214000127AD30701D19207F3D52A68521C2A606C
:102150008A42EEDD2E602070EBE730B41DC8624984
:1021600081E81D00082130BC012003F049B82DE9A9
:10217000F0415B4800240068C17BC90732D05B494D
:10218000564E27460978C90727D0DFF84881012431
:1021900098F8001002290BD004290BD0857C00F0A0
:1021A000D3FC012808D05248007801280BD00EE05B
:1021B000457CF4E7C57CF2E798F80000042806D0D7
:1021C0000024776006E098F80000022807D07068C5
:1021D000401C70607068A84203DD776002E07760A1
:1021E000F8E700242046A4E72DE9FE4339483F4D97
:1021F000012600783F4FDFF80081032816D004281D
:10220000684610D0002402F0A5FBFFF7B0FF297844
:10221000C90700D0012440EA0401C90716D02E499D
:10222000097801B310E000F02EF812E068460024AF
:1022300002F090FBFFF79BFF2978C90700D001242B
:1022400040EA0401C90701D08DF804603860C8F87D
:1022500000402A480090684602F080FB012806D022
:102260000020BDE8FE8302218DF80410EEE702ABEA
:1022700000220821012003F013F80821012002F0B8
:10228000EEFF0120EDE770B50446002502F062FB89
:10229000FFF76DFF1249C3074FF0020205D009682E
:1022A000C97B89070FD504210BE0104B1B78DB0796
:1022B00000D00225AB0707D50968097A490702D57E
:1022C0000521217100E022710A4908600A48056071
:1022D00070BD0000700210000503100068021000BD
:1022E000E00210008C02100028041000740210009C
:1022F000E80210007C021000780210000B210000A0
:102300001C4808B500210122416002708160C16053
:10231000491E104602F0A3FFFFF76DFE6B46002238
:102320001721012002F0BCFF0098800705D5FFF7B8
:1023300054FD0221012002F092FF0098C00705D051
:102340000121084602F08BFFFFF7F4FC00984007DC
:1023500005D50421012002F082FFFFF770FD0098EF
:10236000C006DBD51021012002F079FFFFF776FDD2
:10237000D4E700007002100032216E4803F096B9D5
:102380002DE9FC5F88466C4905466FF0130208682A
:102390004FF0010AC446037CB0F9167003F00F0435
:1023A000B0F91A30C4F11006B8F1280F15DB8B46CE
:1023B0004FF00009C18ACDE90019838A28223C2107
:1023C000604601F0EEFF07B2DBF800002822418BE7
:1023D000CDE90019038B3C2118E008F1140CBCF185
:1023E000140F17D84FF00109C18ACDE90019838A6B
:1023F00093460021404601F0D4FF07B24E48002129
:102400000068428BCDE90029038B5A46404601F013
:10241000C8FF03B24948DFF81CC1006881460AE0E2
:102420003CF9101035F9102001EB0708904515DB39
:10243000C91A914212DC401EF2D2BAF1000F0DD03F
:10244000494609E03CF9112035F91100624300FBCF
:10245000062000112CF81100491EF3D2BDE8FC9FA4
:1024600070B514460D46C00716D000F06DFB00286D
:1024700012D131480068C07B800703D5304800780E
:10248000042804D021462846BDE8704078E7284655
:10249000BDE8704000F001B870BD2DE9F04F26494D
:1024A000284C4FF0010E0A68DFF888B094F900401C
:1024B000117CB2F916A001F00F0692F86D10C6F16A
:1024C0001008B2F91A900B4614E093FBF1F7C3EB36
:1024D000440501FB1737EDB2FFB23BF9155030F957
:1024E000177005EB0A0CBC4522DBA5EB0905BD42C4
:1024F0001EDC5B1E012BE8DABEF1000F18D0DC46B3
:1025000014E092F86D50C1EB440391FBF5F705FB25
:102510001715EDB2DBB230F915703CF91350754365
:1025200007FB08552D112CF81350491E0129E8DA34
:10253000BDE8F08F523C0120E0021000A80210001C
:10254000A4021000A502100070B5FA4C002532213B
:10255000A4F807506572F84803F0A8F8F64A00207E
:102560006FF00041503A42F82010401C1428FADB6A
:10257000F14A0020323247F6FF71CB4302F11406D4
:1025800022F8101026F81030401C0A28F8DB65707D
:102590002571E5706421E94803F088F8E748642173
:1025A000643003F083F86571A57170BDF0B4E44C3C
:1025B00000231A462478022C02D0F0BC184670473B
:1025C000E04B1C68E04B1E6874B900230AE030F948
:1025D000134096F8C950AC4201DCEC4201D501220F
:1025E00002E05B1C8B42F2D396F8B710F0BCD148E6
:1025F000093000F010BA2DE9F84F8246D248002683
:1026000047F6FF780468B346354694F8B100B4F84D
:10261000BA904307B4F8BC7094F8B8006FEA080C9D
:1026200005D5884222DC94F8B9308B421EDB884203
:1026300008DC94F8B900884204DBB4F8BF90B4F821
:10264000C17008E094F8C8004042884203DBB4F847
:10265000C390B4F8C570B849088810B100208E4600
:1026600013E032225146B44802F0A1FFBBE03AF930
:1026700010103EF810300E44C91A0BB2984500DD18
:1026800098469C4500DA9C46401C9042EFD3A949ED
:10269000A94A88783232009022F8108000981432CB
:1026A000A2F1960322F810C04A7800209E4643F813
:1026B0002260C0F114011144142391FBF3FC03FBCD
:1026C0001C180A315EF828C091FBF3F803FB1813BD
:1026D000401C5EF823100A28ACEB01010D44E8DB36
:1026E0009449C87810B1012804D007E04D4505DDB4
:1026F000012002E0FD4201D50220C8700A2095FBAE
:10270000F0F38E4D4879002725F81030401CC0B2F8
:102710004871322800D34F71C8788C46022844D1C2
:102720009CF80480B8F1280F3BD247F6FF73DFF81E
:102730000892D943002009F146097F4D323535F919
:1027400010509D4200DA2B4639F910508D4200DDC1
:102750002946401C0A28F0DBC81A784D9CF8061060
:102760006435634625F81100491CC9B28CF806107F
:10277000322900D39F7194F8BE1088420CDC1F717F
:102780004FF0010B8CF803700020714641F8206077
:10279000401C1428FADB08E008F101008CF8040062
:1027A00003E08CF804708CF8037000986546401CB8
:1027B000C0B28CF802000A2800D3AF70521CD0B20D
:1027C0006870142800D36F70322251465A4802F0C4
:1027D000EEFEE97839B194F8E307DB2803D114223F
:1027E000552001F091FB5846BDE8F88F2DE9F04FD8
:1027F0008FB08346544A00200E9012688846BBF979
:10280000041092F8B520914250DDBBF906209142A8
:102810004CDD00244FEA58000D90DFF830914FF066
:10282000FF3A2746264625463421684602F060FFD7
:1028300042465946684601F095FD434900206B46E3
:102840000A681BE033F91010B0EB580F08D292F869
:10285000B6C0614511DC761C2144F6B20CB20CE026
:1028600092F8B5C0614508DD6D1C0F44EDB23FB272
:10287000494502DD89460FFA80FA401C4045E1D304
:10288000BAF1030F0BD10D98864208D1854206D1CB
:10289000002C00DA6442BC4201DA01200E90254887
:1028A00092F8B71008300E9A00F0B5F80FB0BDE8F6
:1028B000F08F2DE9F05F8346994690468A460024C2
:1028C00002200A9E02F04DFD1F4F1A4D3A6892F801
:1028D000B000C00720D0A4466146604608E038F941
:1028E000103092F8B340A34201DD491CC9B2401C2C
:1028F000B042F4D3B14201D14FF0010C0D4892F82F
:10290000B4106246C01D00F086F80446012801D0CC
:1029100014B130E0102032E0386890F8B000800741
:1029200018D531465046FFF761FF044601280FD005
:1029300084B120E080021000880410004E3801208D
:102940000503100098021000E00210000080FFFF55
:10295000112014E0386890F8B00040071AD53648C6
:102960000078B8B1324649465846FFF744FE04465F
:10297000012803D074B1012C02D005E01220287088
:102980000020A5F807006872022002F005FD20462D
:10299000BDE8F09F386890F8B0000007F4D572B237
:1029A00049465046FFF702FE04460128ECD11320A9
:1029B000E5E770B50646214D0C78002008702868C0
:1029C00090F8B100C00710D0022002F0CAFC1C48E9
:1029D0003146006842001B4802F0E9FD1A48012117
:1029E0000170022002F0D8FC09E01848016841F0AB
:1029F000010101604FF40061002002F001FC286831
:102A00002246012190F8B100BDE8704000F00103BA
:102A1000052001F07ABB10B500231C4642B10278B4
:102A2000521CD2B202708A4203D90470012300E022
:102A30000470184610BD000005031000E0021000ED
:102A4000A8021000523C01208C021000FC02100071
:102A500010B5F94C012019212070F84802F048FE09
:102A6000F64832211A3002F021FEF44832214C306F
:102A700002F01CFEF1490020083948602061E06046
:102A800060704FF4C8706061BDE810404FF49671FB
:102A9000EB4802F00BBEF0B5EA48EB4C01220168AE
:102AA0000020206060602081C4F80A00C4F80E0095
:102AB0006082E64801F13F0301F147060778E448E8
:102AC0000078384303D1E348007800B10222DFF8F0
:102AD00078C300200CF10A0C0EE033F81050554377
:102AE00024F8105033F8105016F800E0A5EB0E054E
:102AF00055432CF81050401C91F86C508542ECDC8A
:102B0000002F0AD0D4480078002806D1CB4831F8ED
:102B1000632F0838028089784180F0BDC948006879
:102B200090F8801069B1490010F88C2F521C407841
:102B30004A43C2EB022100F01F000141BE48C180A0
:102B400070470121F0E77047BB480069002800D0BA
:102B5000012070472DE9F04FB74C4FF0010A0AFAF7
:102B600001F5E468DFF8D4B22540BA4CABF1080BAC
:102B7000DDE909E72678B54C91464FF0000CBBF82B
:102B80000080247862460AD024B1BBF80220A8EB6A
:102B9000020292B2012F0AD04CB146B10BE00CB147
:102BA00006B142460FB904B12EB9A74A01E0A64AC0
:102BB0000A3232F81120A349096891F83A10CC077B
:102BC00030F919102ED0BEF1010F07D030F91340A3
:102BD0008C4200DC0C4694422BDC30E0002906DD00
:102BE00030F91340002C02DD0C4424B204E030F92B
:102BF00013408C4200DC0C4655EA07060BD0002D32
:102C0000E9D0002FE7D19142E5DA30F91300904284
:102C1000E1DA0024DFE79142DDDC30F91300904275
:102C2000D9DCF6E775B1914209DA30F91300904228
:102C300005DA0AFA09F00AFA03FC4CEA000C6046CD
:102C4000BDE8F08F9142F4DC30F913009042F0DCE3
:102C5000F5E72DE9F04115460024621E794E8EB04D
:102C60008046012941D13421684602F041FD7B4F65
:102C7000414668463A6801F075FB397840F6FF72C4
:102C800068462B6800F017FC6B49024628680B7BEE
:102C900020EA0303DB0708D03368B3F84F309342D0
:102CA00003DD20F001000124286083070BD50B7B96
:102CB0009B0708D43368B3F85530934203DA20F009
:102CC0000200A41C286043070FD5097B49070CD4D8
:102CD0003168B1F85730934203DCB1F85910914292
:102CE00003DA20F00400241D2860306890F8E30720
:102CF000DB2808D1002C06D00EB02146BDE8F041FB
:102D0000FD2001F001B90EB0BDE8F08101460020C0
:102D10008A0700D0012011F00C0F01D040F0020012
:102D200011F0300F01D040F00400704730B411783A
:102D300089073DD5B0F90430B0F906108B4237DD74
:102D4000002B00DA0023B0F90040002C00DA002448
:102D5000B0F90850002D00DA00252C44C4EB4303E1
:102D60001BB2002900DA0021B0F90240002C00DA81
:102D70000024B0F90A00002800DA00202044314C79
:102D8000C0EB410000B22168B1F84D10994201DC5E
:102D900081420DDD00211160216891F8E317DB29E4
:102DA00006D140EA0342012130BCFC2001F0ACB85E
:102DB00030BC7047F0B50A680023002A1BD0214CB4
:102DC00003260022246894F85F50540024B230F99E
:102DD0001470AF4205DC00EB4404B4F90240AC428D
:102DE00001DD5B1CDBB2521C12B2B242EDDB032BE5
:102DF00001D100200860F0BDFCB50C460125CDE9ED
:102E000000540746052304220221FFF7A3FECDE963
:102E1000005406460022012311463846FFF79AFE69
:102E2000CDE9005406430323022201213846FFF76F
:102E300091FE3043C0B2FCBD8C021000203901204D
:102E400000EC0120E0021000E2041000043C01202C
:102E5000E80210000503100004031000A80210008F
:102E60002DE9F0410C4601463222FE4802F09FFB5C
:102E7000FC483222FC49323002F099FBF9483222F8
:102E8000FA49643002F093FBF849F64832223231B5
:102E9000963002F08CFBF54A0020FF23223A4FF0D7
:102EA000010E5668F24A0746EE49156814E00EFA1C
:102EB00000F2224201EB400C02D0ACF8C83001E035
:102EC000ACF8C870324201EB400202D0A2F8FA30EE
:102ED00001E0A2F8FA70401CA842E8D314E72DE9FB
:102EE000F843E44C8046E148894600252778257060
:102EF0003221963002F0DAFB17B1B8F806002081D3
:102F0000DD4EDB4C306890F82A10C9070AD00097D4
:102F100090F82B00414600F00F03208802B2D348FE
:102F200001F060FB022002F01CFA2088CF4900B2B9
:102F300000904B46CC4A01F1960001F08FFA022036
:102F400002F02AFAC94932229631A1F1320002F088
:102F50002EFB3068C94FC07B000714D5C8480078E5
:102F6000012810D1387870B9C648007858B1208847
:102F7000BE4900B20090C448963102680846938E5C
:102F8000243201F050F92068B84942009631A1F18D
:102F9000640002F00CFBBD493878097808432FD152
:102FA000306890F82A00400707D5B049227864318C
:102FB000012301F1320000F0ABFA306890F82A10DA
:102FC00089070BD590F86D100091A84990F86C30E6
:102FD00090F82C209631084600F01AFAA3493222C4
:102FE0009631A1F1320002F0E2FAA04A20683232B2
:102FF00000904B4602F132014046FFF75AFC05466D
:103000002846BDE8F8832DE9F0410025984B064697
:103010002C46681E2A46AE46DFF858C21F680CE0F0
:1030200036F912308B4202DA0B44002B04DC012506
:1030300036F9124050B203E0521CBA42F0D3A5B1A7
:103040009CF80110491CC9B28CF8011032290ED924
:103050008F4A8CF801E001211160C3B2E2B2C4F3DF
:103060000721ED2001F051F801E08CF801E028463D
:103070004AE6814A10B5126804460020128C891A6B
:103080000BB27B49096806E034F911209A4201DC51
:10309000DA4200D50120491EF6D210BD70B5764D3A
:1030A000024600242868C07B40071CD51046FFF765
:1030B000E0FF012817D1FDF7A9F9764C206840F010
:1030C00002002060FDF7A0F94FF40041002002F05B
:1030D00097F8286822780121C07BC0F3800307207D
:1030E00001F013F80124204670BD30B56149624BF0
:1030F0000022CD681B68002D14464FEAC07505D02C
:103100007DB185070DD58D782DB10AE04DB18507CC
:1031100007D58C7005E001258D700C7193F89750E0
:10312000CD7010B18C7834B901E08C700C7102460E
:1031300093F89700C870104630BD10B54D4CA0787C
:10314000002805D0E07820B1401EE070207910B949
:1031500010BD01202071454803212238007901F07B
:10316000FFFA0020A070207110BDF0B54A4C414F0D
:103170000E4620780025A8B1B6F90600B7F9081068
:10318000081A00D540423C4900B20968B1F8601005
:10319000814207DA00204149207002200125087091
:1031A000FFF779FC38782178084301D1F08838811D
:1031B0002846F0BD2DE9F04704462C48DFF8B490CE
:1031C00022382A4F4568D9F81000002384EA000805
:1031D00029484FF0010A1A3F066820E00AFA03F076
:1031E00010EA080F10D0204220D023B1012B02D0CA
:1031F00096F83DC006E05FEA817C05D05FEAC47CBA
:1032000096F83BC007F803C017F903C0BCF1000FE4
:103210000FD0ACF1010C07F803C05B1C1BB293424A
:10322000DCDB2846C9F81040BDE8F08796F83EC0C0
:10323000E8E7204201D00543EFE78543EDE72DE9BC
:10324000F34F81B00B4D00240094B5F9061001989E
:10325000FFF7D9FE012843D0A846B5F9061001981A
:103260001EE0000000EC0120523C01203A39012010
:10327000A80210008C021000E0021000E80210000A
:10328000043C012005031000E4021000E9021000D4
:10329000F40210000003100006031000800210006A
:1032A000FFF7FCFE01282BD0DDE90101FFF717FE37
:1032B000044601282CD002F0DBFA012828D0B44AB9
:1032C000DFF8D0A2B1481060DAF80010B24FB34E68
:1032D000C97B090723D5B249097801291AD01EE014
:1032E000B048006801280AD168694FF00051401EBB
:1032F000686111F8350F05D040F00F00087000200C
:10330000BDE8FE8F20F002000870A7480460FDE7CA
:103310002046F5E7397811B99C493239116030609F
:10332000002191461068FFF767FD050006D0387848
:1033300020B901213068FFF75FFD05402846FFF7FF
:10334000E5FC009004216846FEF764F8974900F018
:10335000FF0B38780978084323D1DAF80000554686
:1033600090F83A00400704D56A4659463068FFF79E
:1033700070FC0098A8B1286890F83A00800706D53C
:103380006A4659463068FFF7D1FC009848B1286872
:1033900090F83A00000704D56946D9F80000FFF715
:1033A00009FD03224646D8F80C100098FFF702FFEB
:1033B00007460199FFF7D9FE744D863DA8B1002458
:1033C0006C602046029900F0D0FE2879214601F079
:1033D000C7F9012476480078042803D0DDE90010FD
:1033E000FFF73EFD6868F06092E7686887420CD09E
:1033F000F8B26F60FFF779FE07462879029900F06E
:10340000B4FE2879394601F0ABF9FFF796FEE1E703
:103410002DE9FF4F9146864600250D9F46E005FBAE
:1034200007F00199012247F6FF7C01EB40066FEAA5
:103430000C040EEB400B13460021C9F1000A16E004
:1034400036F9110048450FDA50450DDD844500DDA1
:103450008446844200DA0446002802DA4FF0000273
:1034600002E001DD4FF0000301F1010189B2B94230
:10347000E6D352EA030009D012B1012A04D004E0D5
:10348000012B02D1204601E023B1002041000BD0E6
:10349000002107E06046F9E736F81120121A2BF8F0
:1034A0001120491CB942F7DB6D1CADB2039885426F
:1034B000B5D3BDE8FF8F2DE9F0410024491E174622
:1034C0008646CAB2A44626462546D80701D002221F
:1034D0000DE098070BD50124032208E03EF9140003
:1034E000604502DD00FB04660544641CE4B29442BE
:1034F000F4D985FB012386FB070102F034F800288C
:1035000000DA0020791E884200DD084600B2E5E4BA
:103510002DE9F04F00259B469AB0531EDFB22C4692
:103520002B460DF1340AE94611E031F913603544B8
:103530005E1CB44695FBF6F629F81360FE1A5B1C78
:1035400031F91680444494FBFCFC2AF816C09342DF
:10355000EBDBBBF1010F01D1921ED2B24C465546B6
:103560000FE034F9123035F91260334403EBD373B2
:103570005B101BB2002B04DD31F81260F31A20F847
:103580001230521EEDD21AB0BDE8F08F9E390120E4
:10359000BC021000E0021000E8021000B8021000A7
:1035A000043C0120F40210005C090022E902100032
:1035B00070021000384808B50021C1608160416088
:1035C00001210170354914200870FFF741FAFEF718
:1035D000D3FEFEF7B9FFFFF7A1FA6B4600220121E7
:1035E000022001F05DFE0098C007F6D00121022004
:1035F00001F035FE00F001F8EFE770B5002503207B
:1036000001F0AFFE00F024F8234C244E207BC007CD
:1036100005D096F900102069FFF711FE0546A06855
:1036200058B1022001F09DFE96F900202169A068A2
:10363000FEF716FF022001F0AFFE012D03D118495D
:103640002069FFF7B6F9BDE87040032001F0A4BE81
:1036500070B5114C134DE068B5F90C1080EA010209
:10366000D20708D0C90702D0FFF7F2F903E0C0077C
:1036700001D0FFF768FAB5F90C00E0602869A06096
:10368000A868606007481630206128782070287D7F
:1036900060700548606170BDA4021000F80210005F
:1036A000800210005C0510006C390120094C0020DC
:1036B0002060401C2060FDF770F800F047FEFCF72A
:1036C0003FFF08B9FDF725FFFCF784FD01F088FBFB
:1036D0002068EEE7C0021000E04900200860E049E1
:1036E0000860E04908607047D0214DF6C062BA20FA
:1036F00000F021BC70B54FF40063984202D2DA4C5E
:10370000246807E0A0F5805080B24FF480539842BF
:103710000CD2D64C85189D4200DD1A1A002303E016
:10372000CD5C1E185B1CA5559342F9DB70BDB0F54E
:10373000805F04D20A460146CB48006808E0B0F535
:10374000FE5F07D3A0F5FE5080B20A460146C74887
:1037500000F00EBC704700F0A0BF10B54FF4005150
:10376000002000F06EF90023BDE810401A4619460B
:10377000032000F0CABC10B54FF48041002000F0D7
:1037800060F90023BDE810401A461946042000F0F5
:10379000BCBCB2490A6882430A600221012000F0E1
:1037A00050B9AE490A6802430A600221012000F0C4
:1037B00048B9FDF78EB9FDF767B910B5C00711D04C
:1037C000AB4800230222016841F0010101600121A0
:1037D000052000F09AFCBDE810404FF40061002085
:1037E00000F02FB910BD10B50324FCF70FFEA1485F
:1037F0000460FCF709FE002301211A46084600F088
:1038000084FCBDE810404FF40031002000F019B9ED
:1038100010B5002301221946104600F076FCBDE8E1
:1038200010404FF48051002000F00BB9042101201A
:1038300000F007B98C4A904B0128126892F8E327F0
:1038400009D002280CD0882A09D1197800231A46F9
:10385000172000F05ABC882AF7D0087818707047F3
:10386000882AFCD148781870EFE77E4A00230128A7
:10387000136005D1087810211060012000F0E1B834
:1038800070474FF48021002000F0DBB84FF4002196
:10389000002000F0D6B874480021006890F8680055
:1038A000C00711D075480068827A12B1FF2A03D090
:1038B0000AE0C27A1AB107E0C27AFF2A04D196213F
:1038C0008172A521C172012100231A46102000F047
:1038D0001CBC6A4800210B4600680A468172C1720E
:1038E000202000F012BC10B50978654C002031B1E1
:1038F0000121217063490870FFF7CDF800E02070C6
:103900000120FFF75AFF00232178BDE810401A4636
:103910009A2000F0FABB10B5594C2278D2B9594A16
:103920001278BAB1584A042809D000201070002338
:1039300021781A469F20BDE8104000F0E6BB534BAB
:103940000888188048885249088001201070FFF7C5
:10395000A2F8ECE7494A00EBD070136820F00102AE
:1039600003F1340001F023FE00231A4621789C2045
:10397000E1E7434A1278002A0BD0012809DC3F48CE
:103980000978002300681A4680F83A109D2000F05C
:10399000BCBB704770B53A4C2278A2B1374D00EBF2
:1039A000D07626F001022B6803F1240001F0FFFD20
:1039B00029687008002348842178BDE870401A46C1
:1039C0009B2000F0A2BB2F480078002811D1264B85
:1039D000304A314C1B6808E031F8105022F8105082
:1039E00031F8105024F81050401C93F86C50854268
:1039F000F2DC70BD70B5214A4D78431E14680A7818
:103A00001D445434202D02DBDBB2FF2108E0A31853
:103A1000421E1846491C01F0CAFD00231A46012126
:103A2000BDE87040992000F070BB30B41B4C00B171
:103A3000087820700023C1B230BC1A46A32000F0E1
:103A400064BB38B50C46054601F0DAFB69462846EA
:103A500001F015FC009A2242F8D138BDEC021000AA
:103A6000F0021000F4021000E00210004C000120EF
:103A7000FC02100000031000F8021000E402100025
:103A8000E8021000043C0120040310001839012052
:103A90001A390120E2041000EC041000E9021000C1
:103AA00010B52021664801F001FE6548FDF718F8C1
:103AB0006349401E11F8012BA2F190031F2B01D87E
:103AC000604A05E0A2F1C0030F2B06D85D4A8032A0
:103AD00052F82320BDE810401047B82A21D00DDC51
:103AE000B02A13D0B22A27D1032825D108888A7892
:103AF000BDE8104040BA1146FFF719BEFB2A17D0A7
:103B0000FC2A19D1BDE81040FFF735BE022813DDAD
:103B100031F8022BBDE8104053BA821E1846FFF759
:103B2000E9BD022808D10888BDE81040FFF713BEA0
:103B3000BDE81040FFF711BE10BD0120FFF731BEF8
:103B40000120FFF726BE10B5FEF7FEFCBDE81040D1
:103B50000120FFF732BE00F053BA3B4810B50178A0
:103B600009B10221017039483949006891F90030E2
:103B700090F824219A420CDD90F81C0191F9001074
:103B8000884206DAFEF7E0FCBDE810400120FFF7AE
:103B900014BE10BD2C480178002903D00321017008
:103BA000FEF779BF704770B52A4D284C0020287069
:103BB00020680078A52802D0012000F0C9F840F262
:103BC000FF112068FDF70CFC2168D1F8FC17814239
:103BD00002D0022000F0BCF840F2FF311E48FDF791
:103BE000FFFB1D49D1F8FC1F814206D020680079F7
:103BF000800702D4032000F0ABF818480078810752
:103C00004FF0010001D5287070BD0F490870FEF714
:103C100042FFBDE870400120FFF7CFBD0A4910B553
:103C200000200870FEF737FF08480068007A800718
:103C300001D5FFF7FBFDBDE810400120FFF7BDBD3A
:103C4000F6041000C85C000005031000E00210003C
:103C5000F8021000060310004C0001201C3901205E
:103C600008B5FFF739FD00F0AEF91B4C206800796C
:103C7000800701D5FFF7B7FD20680079C00701D0A4
:103C8000FFF75BFF2168C87B00070DD511F86C0FAB
:103C90004978484300F092FA104900231A46087008
:103CA0000146C02000F031FAFEF7F5FE01216B4617
:103CB0000022032001F0F4FA0098C007F6D0FFF7C5
:103CC000EFFE0121032001F0CAFAFCF71DFFEDE72A
:103CD0000121032001F094BAE0021000043C01200D
:103CE0002E4C2D4AC4E900210168A1604168E160C1
:103CF00081682161C16861610169A1614169E16116
:103D000081692162C069606204F12800FDF711FC3D
:103D100001F0DFFB606400F035F82049204AC1E97A
:103D20000020704710B501284FF0000205D0014671
:103D3000BDE81040022000F0FEB80121022000F092
:103D4000FAF800F01FF8012801D10220EAE77047D5
:103D500010B5044601460022032000F0ECF8012CC7
:103D600001D0022C01D100F00DF810BD0022014657
:103D7000062000F0E0B801460022072000F0DBF842
:103D800000F000F8FCF709FD4FF0005010F8351F67
:103D900021F002010170FEE7AF0550FA00EE0120AC
:103DA000BA0110AB77B585B00E46BDF81440154684
:103DB000200A40EA0420ADF814004F48BDF8141062
:103DC00000240180A0F58070CDE900044B480294E6
:103DD000039400681346484AC0790221FCF701FEAB
:103DE00008B02A463046BDE87040454901F0DFBBC7
:103DF00017B581B00B46BDF804001446010A41EA2C
:103E00000020ADF804003C48BDF8041020F8021B67
:103E1000194601F0CCFB0020009038480023364AB8
:103E20000068A11CC079FCF7ABFD1FBD77B585B05C
:103E30000E46BDF814401546200A40EA0420ADF8AD
:103E400014002D48BDF81410002401802C48CDE941
:103E500000042A480294039400681346264AC07955
:103E60000221FCF7BEFD08B02A463046BDE870408E
:103E7000234901F09CBBFCF773BB08B50020ADF8EB
:103E8000000002226946FFF78DFFBDF8000008BD63
:103E900000B587B0002201210720FCF787FE07202C
:103EA00001F0D4FC00204FF4FA7100BF401C88429E
:103EB000FBDB072001F0D3FCFFF7DFFFA0F5844117
:103EC0000E3902D00120FFF72DFFAFF2DB00019089
:103ED000AFF22F100090AFF2AB000290AFF269008A
:103EE00003900848049040F28F20ADF81400684613
:103EF000FCF7FCFE07B000BD043B0120E00210000F
:103F0000043A0120030500001CB5DB238DF80030C6
:103F10008DF801008DF80210100E8DF80300100CC2
:103F20008DF80400100A8DF805008DF8062068460B
:103F300000F032F91CBD1CB50F238DF800308DF850
:103F400001008DF80210080A8DF803008DF8042096
:103F5000100A8DF80500100C8DF80600100E95491A
:103F60008DF80700012008706846FCF7DCFD1CBDD9
:103F70002DE9FC41002706460097122015460C4605
:103F800001978DF800001AE0200A8DF80100C4F3B3
:103F90000B008DF80240315C30448DF803104178FD
:103FA0008DF8041081788DF80510C0788DF8060022
:103FB0008DF80770684600F0EFF8241D2D1F002DC6
:103FC000E2DCBDE8FC811CB500207B49009001903B
:103FD000096810234A7889788DF800308DF804003C
:103FE0008DF801008DF805208DF802008DF806107F
:103FF0008DF803008DF80700684600F0CDF81CBD71
:1040000070B588B000240094142001948DF800004D
:10401000FDF7B0FA8DF80100F2208DF80300664E2E
:1040200065208DF804003068624D41788DF80510E8
:1040300080788DF80600287880018DF807006846A2
:1040400000F0AAF80094152001948DF80000306863
:1040500090F8EC178DF8011090F8ED178DF802101C
:1040600090F8EE178DF8031090F8EF078DF8040024
:10407000287880018DF80700684600F08DF80094DC
:1040800002A80194FDF787F91B208DF80000029823
:10409000000E8DF801000298000C8DF802000298C5
:1040A000000A8DF8030002988DF804008DF8054091
:1040B00004988DF80600287880018DF8070068467E
:1040C00000F06AF800941C208DF800000398019419
:1040D000000E8DF801000398000C8DF80200039883
:1040E000000A8DF8030003988DF8040005988DF8F8
:1040F000050006988DF80600287880018DF80700E5
:10410000684600F049F808B070BD1CB52A4C246818
:1041100094F8E247A40710D50024019400941624D3
:104120008DF800408DF801008DF802108DF8032005
:104130008DF80430684600F02FF81CBD1CB5002334
:1041400000930193E1238DF800308DF80100080AF7
:104150008DF80200100A8DF804008DF803108DF818
:104160000520684600F018F81CBD1CB5124A1268FC
:1041700092F89320D2070ED0002200920E230192D3
:104180008DF800308DF801008DF806108DF80720AD
:10419000684600F001F81CBD10B50446012001F08E
:1041A000E0F82046FCF7BFFCBDE81040012001F01C
:1041B000F3B80000C4021000E0021000F0B523497B
:1041C000074601200A68518C59B32149096891F8C2
:1041D000693092F83A108B4202D009B1FF2920D100
:1041E00002F1340602F12404B51C00214FF6FF7CD5
:1041F000383208E034F811300BB1634501D10020AA
:1042000003E0491C89B2B942F4D3318809B1FF29CE
:1042100000D10020298821B1FF2902D012889142C3
:1042200000D20020F0BDF0B50024059E0AE031F96F
:10423000145032F814705D4395FBF7F520F81450D4
:10424000641CA4B2B442F2DBF0BD0000E402100032
:10425000E002100070B54A21304801F027FA2F4CD7
:10426000A6202F4D20804FF265206080286841787D
:10427000217180786071FDF779F9E080FFF7FDFD2D
:104280002081286890F86C10217790F86D10617784
:104290002449E18324492184244961842449A18754
:1042A0002449A1842449E18424492185D0F8FC17BC
:1042B0000A0C6285A185B0F83F10E185B0F8411085
:1042C0002186B0F843106186B0F84510A18690F8B9
:1042D000741001F0030284F83620C1F3011184F850
:1042E000371090F8681001F001012187144909681E
:1042F0004A8952BA628701F12202E2873232A4F877
:10430000422090F8690004F8440F91F83A00607078
:104310000C4824F8020F0C48608070BD000001209A
:10432000E0021000063C01203A3901206C390120DE
:104330009E390120523C0120C00001201C3901207F
:10434000E4021000183901201A39012010B5FCF7D9
:104350005DF8FDF7CCF808B1FDF7C3F8BDE81040F3
:10436000FCF752B830B501230CE000EB430531F8FF
:10437000134025F8024C01EB430434F8024C20F8BA
:1043800013409B1C9342F0D330BD10B5FCF73EF8B0
:10439000FDF7ADF808B9FDF79EF8BDE81040FCF751
:1043A00033B8F0B5851ADDE905471E1B75438E1A33
:1043B000012F02D0904206DD0BE0904201DC18464E
:1043C000F0BD884201DB2046F0BD95FBF6F0181ADF
:1043D000F0BD8842F3DA95FBF6F02044F0BD2DE9FC
:1043E000FC4F04468F480B4600260768354607F504
:1043F0008A7207F58E7C125707F5927807F5967149
:1044000007F59A7907F59E7A07F5A27B184607F516
:10441000A6779A4200DD10460957994200DA08460D
:1044200082420ADC1CF90430834206DB194619F982
:10443000043001251AF9044008E018F904208242EA
:1044400009DC814207DB3B571BF90440CDE90045FD
:10445000FFF7A7FF46B23046BDE8FC8F2DE9F84FC5
:10446000894670490546DFF8C0A108689B4690461A
:1044700090F8E307882808D12A68CAF800206A68FB
:10448000CAF80420AA68CAF8082000245AE067483D
:1044900039F81410634B076838F814000126081A1D
:1044A00025F814001868243790F8E317882906D1F6
:1044B00039F8142038F81410511A2AF81410C07B57
:1044C000C0063DD55A480078D0BB5A48007801282C
:1044D00036D15948007898B3A0B25946FFF77FFF0C
:1044E00001465048006890F8E307882805D15348F2
:1044F00080F830B2204480F831120AEB4400818108
:10450000F1B135F9140064225043C1F1640290FB0B
:10451000F2F000B2002802DA0026404200B237F87A
:104520001420824205DC821A4A43642192FBF1F195
:10453000401A25F814001EB980B2404225F8140034
:10454000641C24B20A988442A1DB3648006890F8C3
:10455000E307882835D12968CAF818106968CAF8AD
:104560001C10A968CAF82010062000902F482E4978
:104570000268183101F10C00938E2432FFF753FECC
:104580002E4F2F4E6FF0130530883D54401C308065
:104590000024A0B22946FFF722FF3188641C24B210
:1045A0007854491C3180062CF3DB6D1C6DB23C2D18
:1045B000EADB3088B0F50C7F07F800B001D30020AB
:1045C0003080BDE8F88F70B5002408E031F8145051
:1045D00032F81460AD1B20F81450641C24B29C42C5
:1045E000F4DB70BDF0B4049C012C04D01BB1C3F10A
:1045F0001006002412E0F0BC520000F0D8BF30F9E1
:10460000145031F914705D4307FB0655EF1705EBA5
:1046100017752D1120F81450641C24B29442EEDB5F
:10462000F0BC7047E0021000BC3E0120E402100024
:10463000E8021000043C012005031000843C012026
:10464000C60210000FB42DE9F05F0025DDF874A05C
:104650008B4681462E464FF0010808FA06F70024E3
:1046600007EA0B076FB108FA04F010EA090F08D047
:10467000324621460C9800F0A5FA0AF805006D1C98
:10468000EDB2641CE4B2052CECD3761CF6B2052E18
:10469000E3D3BDE8F01F5DF814FB10B504465021CC
:1046A0002B4801F003F82B4A1178491C1170A00522
:1046B00004D5BDE81040264800F001B810BD2DE932
:1046C000F041044690B0A52020704FF40070A4F88B
:1046D000010000F07EF9207100F076F9607100F0C1
:1046E0006EF9804600F066F905461B4800680179BE
:1046F000552904D1D0F8050020F07F40A060174E66
:10470000392206F1740796F8B000207304F13000E6
:104710000F90391D684600F08FFF00222946404661
:10472000736FFFF78FFF04F110000F903922391DCE
:10473000684600F081FF012229464046736FFFF76B
:1047400081FF04480078E07010B0BDE8F0810000FF
:1047500000800120C8021000E40210004C0001207B
:1047600070B5704E05460C46306890F8940001070D
:1047700008D5E10700F0070002D001F067F801E07A
:1047800001F06DF8306890F89410080608D5A0077D
:10479000C1F3021002D501F059F801E001F05FF811
:1047A000306890F89500010708D5690700F0070008
:1047B00002D501F04BF801E001F051F8306890F8B3
:1047C0009610080712D55848007878B157480078F5
:1047D00060B95748007848B95648007800284FEA31
:1047E000847009D000280FD1A8070DD1BDE8704012
:1047F00001F0070001F033B80028F5D0BDE87040A3
:1048000001F0070001F022B870BD10B5454C2068DA
:1048100090F89400010715D500F0070001F01FF88B
:1048200020680022012190F8940000F00700FCF7B6
:10483000BDF920680022114690F8940000F00700AE
:10484000FCF7CAF9206890F89400010615D5C0F36A
:10485000021001F004F820680022012190F8940071
:10486000C0F30210FCF7A2F920680022114690F86C
:104870009400C0F30210FCF7AFF9206890F895009F
:10488000010715D500F0070000F0E9FF20680022BD
:10489000012190F8950000F00700FCF787F92068E7
:1048A0000022114690F8950000F00700FCF794F9FB
:1048B000206890F89500010615D5C0F3021000F0AD
:1048C000CEFF20680022012190F89500C0F302106D
:1048D000FCF76CF920680022114690F89500C0F3AF
:1048E0000210FCF779F9206890F89600010717D5B7
:1048F00000F0070000F0B3FF20680022012190F8CB
:10490000960000F00700FCF751F9206800221146DC
:1049100090F89600BDE8104000F00700FCF75CB985
:1049200010BD0000E002100005031000E8021000B6
:10493000E90210009002100010B500F001F91B49C7
:104940000020086010BD10B5FFF7E7F9BDE8104082
:10495000FCF7BFB8002101604160704710B50179D4
:1049600099B1134900220A604A608A60CA600F49FF
:10497000D0E90020C1E90120081D00F01FF90B4813
:10498000001D00F0B3F9012010BD002010BD10B5CE
:104990000749064C087020688860201D016804489B
:1049A00088472068401C206010BD0000CC02100029
:1049B00018051000FD48006890F86A007047FB4831
:1049C000006890F86B007047F848006890F86C0039
:1049D0007047F648006890F86D00704770B50400A5
:1049E00004D1FCF776F9F349F1484860F248F34AFC
:1049F000002101701160F24801230360450685F82B
:104A0000EE10F04EA0253560016013602046BDE831
:104A10007040FFF7BCBF10B50446142100F068FEDB
:104A20000020207080206070A020A070FFF7C7FFDA
:104A3000E070FFF7BFFF2071FFF7C6FF6071FFF75F
:104A4000C8FFA071D948E279006810F8771F61F3B8
:104A50008612E27110F80519490861F3C712E27174
:104A6000C18821818168E1600378217C63F30001C2
:104A7000217403785B0863F34101217403789B0878
:104A800063F3820121740378DB0863F3C3012174AB
:104A900003781B0963F30411217403785B0963F342
:104AA0004511217403789B0963F3871121744378BE
:104AB000617C63F30001617443785B0863F3410137
:104AC000617443789B0863F3820161744378DB0867
:104AD00063F3C301617443781B0963F304116174C8
:104AE00043785B0963F34511617443789B0963F371
:104AF00086116174837863F30102E27183789B0805
:104B000063F38202E27183781B0963F3C402E271EA
:104B100083789B0963F34512E271C27862F3C7118F
:104B20006174C1780A09A17C62F30101A174007962
:104B300060F38201A1742046BDE81040FCF76BB918
:104B40002DE9F0419C4800244FF0E02704704470A8
:104B50008470C47004714FF080764FF00108C7F87C
:104B600080619948A02580F80054202297499848F0
:104B7000843700F061FD934808380560954804606B
:104B80008F49091DC1F80080710181F8DE80C7F8E6
:104B9000FC61FE673D229049A020FCF77FFA8E4819
:104BA000743890F8B000FCF77EFA8C48FFF733FFBA
:104BB000BDE8F0418948143000F0D4B87E490020A7
:104BC00008707047844B02EB4202743B03EB820295
:104BD00002EB410110B191F87500704791F8740033
:104BE00070472DE9F041DFF8C4C102460024714D41
:104BF0000127714BDCF80000052912D0042949D0A7
:104C0000FFF7DDFED070FFF7D5FE1071FFF7DCFE79
:104C10005071FFF7DEFE9071BDE8F0411046FCF7E1
:104C20006AB8017A490726D593F903100CE090F889
:104C30006E6007FA01FE16EA0E0F04D0D9701979DA
:104C4000491C197102E0491C0529F0DBD97890F85C
:104C50006A6007FA01FE06EA0E061671577193F9AB
:104C600004606E73491CD97090F86C10B14209DC75
:104C7000DC701C7106E06C7390F86E10117190F886
:104C80007010517190F86F00D070DCF8000090F84F
:104C90007100C0E793F901100CE090F86A6007FA20
:104CA00001FE16EA0E0F04D059709978491C9970CC
:104CB00002E0491C0529F0DB5771597810F86A6F3A
:104CC0008F403E4016714078D070DCF80000491CDF
:104CD00090F86D60967193F902602E73597090F898
:104CE0006C00B04298DC5C709C7095E730B504793C
:104CF00089B0B4B12021684600F0FAFC6D46214627
:104D00003648FFF76EFF354920221431284600F05F
:104D100093FC0025062C10D2DFE804F00F0F060DDF
:104D2000060609B0012030BD2048006890F89000C8
:104D30008DF8110001E08DF81F506846FCF785F8EA
:104D40001D49012008701F480C38056011204107DB
:104D500081F8EE00E5E718480078012801D1FBF75B
:104D6000A8BF7047AFF28B310160114981603231C9
:104D7000C160002101740D49096811F8802F427447
:104D80004A7882744A8882828A88C282CA88028368
:104D90000A8942834A8982830A7B8277497B01F0B0
:104DA0001F01C17741F2883181807047E002100015
:104DB000063C012018051000D80210001005002242
:104DC000901B0022100C022018E000E0885D00001B
:104DD00000000220E01E0022C00001202805100073
:104DE00010B5FCF79CFBFBF7CBFCBDE81040FFF7D0
:104DF000CCBA10B50AF14EFF10BD10B5FFF7F0FFA9
:104E000010BD10B5FFF7ECFF10BD10B5FFF7E8FFC0
:104E100010BD10B5FFF7E4FFFEF75AFF10BD10B547
:104E2000FFF7DEFF10BD10B5FFF7DAFFFBF7AEFBB3
:104E300010BD10B5FFF7D4FFFBF7E6FB10BD10B5B2
:104E4000FFF7CEFFFBF709FC10BD10B5FFF7C8FF59
:104E500010BD10B5FFF7C4FFFBF727FC10BD10B560
:104E6000FFF7BEFFFBF767FC10BD10B5FFF7B8FFFB
:104E700010BD10B5FFF7B4FF10BD10B5FFF7B0FFC0
:104E800010BD10B5FFF7ACFF10BD10B5FFF7A8FFC0
:104E900010BD10B5FFF7A4FF10BD10B5FFF7A0FFC0
:104EA00010BD10B5FFF79CFF10BD7047704710B5DF
:104EB000FFF796FFFBF7A1FC10BD704770477047E6
:104EC000704710B5FFF78CFFFFF745FF10BD704727
:104ED00030B58DB04FF26520FCF727FBFCF7E3FA05
:104EE0004FF400624B494C4800F0A6FB4FF480524F
:104EF0004A494B4800F0A0FBFBF7CCFD0120FBF733
:104F0000E0FDFCF775F90E246846FCF793F9069866
:104F1000C01C65D00698401C64D00698801C61D0E7
:104F20000698C4B22046FCF7EDFAFCF7D4FAFCF779
:104F300025FB3C4C20680078A52802D00120FEF714
:104F400007FF40F2FF112068FCF74AFA2168D1F808
:104F5000FC17814202D00220FEF7FAFE40F2FF3138
:104F60002F48FCF73DFA2E49D1F8FC1F814206D0AC
:104F700020680079800702D40320FEF7E9FEFBF7E2
:104F8000F3FDFBF745FA2948274D016808795528B4
:104F90002CD07020FEF7EAFE2846FBF7C2FAFBF79A
:104FA000B5FC20680079400704D42149002008603E
:104FB000091F0860FEF76CFFFFF7BEFCFBF7F2FB72
:104FC00038B1002211460120FEF7B5FF0120FEF79F
:104FD000A4FEFBF7D0FB0DB0BDE83040FFF715BCD9
:104FE000312000E03020FEF7C1FE9BE7D1F805003C
:104FF00020F07F45D0E710B5FBF708FAFFF768FF10
:10500000FFF728F900F016F8FBF7FEF900F07EF83C
:10501000012010BDF0EF030000F00120F0CF0300ED
:105020004C000120E002100000770100E4021000B3
:10503000841400227FB500F041F81F4D002405EBD9
:10504000441000F11002017F4CCACDE90261CDE9A4
:1050500000230FC800F0DAF910B10220FEF78BFE32
:10506000641C052CEBDB144D0024A03504EB44003C
:1050700005EB800155F820008A68496800F046F980
:1050800010B10220FEF777FE641C042CEEDB0A4D03
:105090000024D03505EBC400416855F8340000F019
:1050A0008FF810B10220FEF766FE641C042CF1DBC1
:1050B0007FBD0320FEF75FBEA85D00001A4910B552
:1050C0000120087019490020086019490860194931
:1050D00008601949086000F07DF900F00FF900F050
:1050E00067F8002010BD10B5124800F024FA1049EE
:1050F00008600E490968884207D00B4800780228EA
:1051000003D1BDE81040FBF739B910BD10B5FFF76A
:10511000EAFF054902200870FBF714F94FF0FF3051
:1051200010BD0520704700000703100008031000A1
:105130000C031000100310001403100070B50D468E
:105140000446C1698068CC2200F0A8FAE169A06831
:10515000084440384FF08071C163216A81630021A7
:1051600041630163C1628162C0E908514FF00B31B4
:10517000C1614FF00A3181614FF0093141614FF057
:10518000083101614FF00731C1604FF00631816095
:105190004FF0053141604FF00431016070BD82690C
:1051A0008168914202D84068FFF783BF70470000D2
:1051B00010B54FF4B4714F4800F09AFA002010BDBA
:1051C00070B5054600EBC5014A4800EB8104FBF7CA
:1051D0000DF90646207828B13046FBF70FF96FF03D
:1051E000010070BD0320207000206560206204F182
:1051F0001C0000F079F93046FBF700F9002070BD83
:105200002DE9F0410F463B49002500EBC00001EBC2
:1052100080042E46FBF7EAF88046206A3843206275
:1052200004F11C00074600F086F90CE0216A026CCC
:10523000114203D000F026F9012600E06D1C29463A
:10524000384600F06EF90028F0D1012E01D1FFF7A9
:105250004AFF4046FBF7D2F80020BDE8F08170B568
:105260000D46244900EBC00001EB8004FBF7BEF8BB
:10527000216AA9432162FBF7C1F8002070BD70B517
:105280000C461C4900EBC00001EB800500202060AB
:10529000FBF7ACF8296A2160FBF7B0F8002070BD7D
:1052A0002DE9F0410D46134900EBC0001E46904623
:1052B00001EB8004FBF79AF807460F480068056485
:1052C000216A294203D104F11C0100F0EDF83846AF
:1052D000FBF794F8FBF78AF8216A29403160B8F1AE
:1052E000010F02D1216AA9432162FBF787F8002050
:1052F000B3E70000641910000803100010B54FF464
:10530000C871324800F0F4F9002010BD2DE9F041D9
:10531000884605462D4900EB8500174601EBC00481
:10532000FBF764F80646207830B13046FBF766F8A4
:105330006FF00100BDE8F08102202070E7611422C7
:10534000414604F10800656000F031F90020206258
:1053500004F1240000F0C8F83046FBF74FF80020B5
:10536000E8E770B5194900EB800001EBC004FBF7DA
:105370003DF80546D4E90701814205DB144804F1F4
:105380002401006800F090F8206A401C2062284642
:10539000FBF734F8002070BD70B50C4900EB8000BD
:1053A00001EBC004FBF722F80546206A08B1401E55
:1053B000206204F1240000F0BEF810B1606A00F031
:1053C00011F82846FBF71AF8002070BDCC1A10001F
:1053D0000803100010B54FF42A71404800F088F916
:1053E000002010BD10B5044690F8380002280BD0FC
:1053F000204600F0A2F8022084F838003849204600
:1054000000F076F8FFF76FFE002010BD2DE9F05F89
:105410008B460646314900EB06109046DDE90AA9A5
:1054200011F820201D461AB16FF00100BDE8F09F71
:1054300001EB8004FAF7DAFF074601202070C4E987
:105440000165C4E90585C4E907A91422594604F198
:10545000240000F0ACF8002084F8370084F838000D
:105460006169E0602061C4E90F1020460C99FFF7E4
:1054700065FEA0602046FFF7B5FF3846FAF7BEFF8D
:105480000020D3E710B5044690F83800022809D070
:10549000204600F052F8022084F8380010492046D7
:1054A00000F026F8002010BD70B5044690F83800D2
:1054B0000D4602280BD1204600F03FF8032084F867
:1054C00038002946204600F013F8FFF70CFE0020B4
:1054D00070BD044800684068704700005C1C100004
:1054E00010031000080310000021016008467047F7
:1054F00030B50A6812B10B46C46B09E0002208609F
:10550000C0E903210BE000BF02F10C03D26812B125
:10551000D56BA542F8DC1A68C0E9032118600020A9
:1055200030BD0068002201E0C068521C8A4201D0F0
:105530000028F9D170470068704702690AB1116804
:1055400031B96FF00400704701F10C02C96839B13C
:105550008142F9D1C9681160002101610846704794
:105560006FF00300704710B54C1084EA530404D563
:105570004042C1F1000138BF491E1B4204D55242CE
:10558000C3F1000338BF5B1E00F0D9F814F0804F60
:1055900004D04042C1F1000138BF491E14F0004F51
:1055A00004D05242C3F1000338BF5B1E10BD032A72
:1055B00040F2308010F0030C00F0158011F8013B30
:1055C000BCF1020F624498BF11F801CB00F8013B17
:1055D00038BF11F8013BA2F1040298BF00F801CBDB
:1055E00038BF00F8013B11F0030300F02580083AB2
:1055F000C0F0088051F8043B083A51F804CBA0E809
:105600000810F5E7121D5CBF51F8043B40F8043B5D
:10561000AFF30080D20724BF11F8013B11F801CB92
:1056200048BF11F8012B24BF00F8013B00F801CB63
:1056300048BF00F8012B704710B5203AC0F00B802E
:10564000B1E81850203AA0E81850B1E81850A0E886
:105650001850BFF4F5AF5FEA027C24BFB1E81850E0
:10566000A0E8185044BF18C918C0BDE810405FEA50
:10567000827C24BF51F8043B40F8043B08BF7047CC
:10568000D20728BF31F8023B48BF11F8012B28BFD1
:1056900020F8023B48BF00F8012B704702F0FF03DF
:1056A00043EA032242EA024200F002B84FF000024D
:1056B0000429C0F0128010F0030C00F01B80CCF124
:1056C000040CBCF1020F18BF00F8012BA8BF20F892
:1056D000022BA1EB0C0100F00DB85FEAC17C24BFE6
:1056E00000F8012B00F8012B48BF00F8012B704790
:1056F0004FF0000200B5134694469646203922BF6B
:10570000A0E80C50A0E80C50B1F12001BFF4F7AFB5
:10571000090728BFA0E80C5048BF0CC05DF804EB97
:10572000890028BF40F8042B08BF704748BF20F805
:10573000022B11F0804F18BF00F8012B704753EA7D
:10574000020C00F069802DE9F04B4FF00006002BB1
:105750001FBFB3FA83F503FA05F424FA05F65E4099
:1057600012BF1643B2FA82F502FA05F4C5F120051C
:105770001EBF22FA05FC44EA0C04203556EA044C0C
:105780004FEA144418BF641C4FF000084FF00009A2
:10579000904271EB030C39D3002919BFB1FA81F79C
:1057A00001FA07F6B0FA80F700FA07F6C7F120070A
:1057B0001EBF20FA07FC46EA0C062037B6FBF4FCB5
:1057C000A7EB0507103F07F01F0BCBF120060CFAE3
:1057D0000BFB2CFA06F644BFB3460026202FA4BFCD
:1057E0005E464FF0000B5BEA060C08BF4FF0010B62
:1057F00019EB0B09ABFB027C48EB0608C01B06FB50
:1058000002CC0BFB03CC71EB0C01C1E70B4602464B
:1058100041464846BDE8F08B13B54FF000004FF00D
:105820000001AFF30080BDE81C40704710B504468E
:10583000AFF300802046BDE81040FAF7C1BC7047C6
:1058400001491820ABBEFEE726000200012181407D
:105850004FF0005010F8352F8A4302707047012135
:1058600081404FF0005010F8352F0A430270704706
:1058700010B50B480A4A007851789278012803D86D
:10588000012901D8012A09D9064B1B6893F8E3378F
:10589000FA2B01D1FEF738FB012010BD002010BD0E
:1058A00087021000E0021000441D0A5D3F1E1D1D0E
:1058B00006080708220F052F200F0F0F020404040B
:1058C0001108031810080808000202020904020C5B
:1058D00008040404000101015A280D7B54282828DB
:1058E000090B090B2D14073E2A141414040605068F
:1058F000170A041F150A0A0A010303030C05021004
:105900000B0505050002020200010102010202036B
:105910000102020302030304000000001B000080D8
:105920002D00008036000000410000805A00000079
:105930006C00000077000080990000808200000069
:10594000B4000000AF000080D8000000C300008059
:10595000F5000080EE000000290100803201000007
:10596000040100001F010080680100007301008035
:10597000450100805E010000B0010000AB01008025
:105980009D01008086010000F1010080EA01000015
:10599000DC010000C70100804902008052020000C3
:1059A000640200007F0200800802000013020080F1
:1059B000250200803E020000D0020000CB020080E1
:1059C000FD020080E6020000910200808A020000D1
:1059D000BC020000A7020080600300007B0300807F
:1059E0004D03008056030000210300803A030000AD
:1059F0000C03000017030080F9030080E20300009D
:105A0000D4030000CF030080B8030000A30300808C
:105A1000950300808E03000089040080920400003A
:105A2000A4040000BF040080C8040000D304008068
:105A3000E5040080FE040000100400000B04008058
:105A40003D04008026040000510400804A04000048
:105A50007C04000067040080A0050000BB050080F6
:105A60008D05008096050000E1050080FA05000024
:105A7000CC050000D7050080390500802205000014
:105A8000140500000F050080780500006305008004
:105A9000550500804E050000C0060000DB060080B2
:105AA000ED060080F6060000810600809A060000E0
:105AB000AC060000B70600805906008042060000D0
:105AC000740600006F0600801806000003060080C0
:105AD000350600802E060000E9070080F20700006E
:105AE000C4070000DF070080A8070000B30700809C
:105AF000850700809E070000700700006B0700808C
:105B00005D07008046070000310700802A0700007B
:105B10001C07000007070080090900801209000027
:105B2000240900003F090080480900005309008053
:105B3000650900807E090000900900008B09008043
:105B4000BD090080A6090000D1090080CA09000033
:105B5000FC090000E7090080200800003B080080E5
:105B60000D08008016080000610800807A08000017
:105B70004C08000057080080B9080080A208000007
:105B8000940800008F080080F8080000E3080080F7
:105B9000D5080080CE080000400B00005B0B0080A1
:105BA0006D0B0080760B0000010B00801A0B0000CB
:105BB0002C0B0000370B0080D90B0080C20B0000BB
:105BC000F40B0000EF0B0080980B0000830B0080AB
:105BD000B50B0080AE0B0000690A0080720A00005D
:105BE000440A00005F0A0080280A0000330A00808F
:105BF000050A00801E0A0000F00A0000EB0A00807F
:105C0000DD0A0080C60A0000B10A0080AA0A00006E
:105C10009C0A0000870A0080800D00009B0D008018
:105C2000AD0D0080B60D0000C10D0080DA0D000042
:105C3000EC0D0000F70D0080190D0080020D000032
:105C4000340D00002F0D0080580D0000430D008022
:105C5000750D00806E0D0000A90C0080B20C0000D4
:105C6000840C00009F0C0080E80C0000F30C008006
:105C7000C50C0080DE0C0000300C00002B0C0080F6
:105C80001D0C0080060C0000710C00806A0C0000E6
:105C90005C0C0000470C0080C90F0080D20F000090
:105CA000E40F0000FF0F0080880F0000930F0080BA
:105CB000A50F0080BE0F0000500F00004B0F0080AA
:105CC0007D0F0080660F0000110F00800A0F00009A
:105CD0003C0F0000270F0080E00E0000FB0E00804C
:105CE000CD0E0080D60E0000A10E0080BA0E00007E
:105CF0008C0E0000970E0080790E0080620E00006E
:105D0000540E00004F0E0080380E0000230E00805D
:105D1000150E00800E0E000047380000833800008A
:105D2000F13A0000EB3A0000993600009936000085
:105D300099360000C137000099360000A5390000EF
:105D40009738000045390000C738000023390000AB
:105D50000B3B0000453B0000633700006737000045
:105D6000F73A0000DB390000993600009737000051
:105D700099360000333800003D38000099360000A5
:105D8000073B000099360000573B0000CD3B000068
:105D9000E53700001B3800009936000099360000F6
:105DA00099360000993600009936000099360000B7
:105DB00099360000993600009936000099360000A7
:105DC0009936000099360000993600009936000097
:105DD0009936000099360000046C00080000047C2D
:105DE00003430001187801001A604002400C0300D0
:105DF0000782000C0D00000000000000985E00000B
:105E000005000000A405100000040000151B0000A0
:105E1000000000000200000001000000EC5E000035
:105E200004000000A409100040060000B122000098
:105E30000000000002000000020000001C5F0000E3
:105E400003000000E40F10000008000065350000AA
:105E5000000000000200000003000000B85E000027
:105E600002000000E417100000010000113C0000D7
:105E7000000000000200000004000000C85E0000F6
:105E800001000000E4181000800000005D360000F2
:105E9000000000000200000000000000C05E0000E2
:105EA0000100000001000000F85E00000100000099
:105EB00002000000045F0000010000000300000079
:105EC000D45E00000100000000000000A45E00009D
:105ED00001000000E05E000002000000145F00000E
:105EE00003000000B05E000054736B5F5353766391
:105EF00000000000456C665F53737663000000008D
:105F0000456C665F436D640054736B5F436D640062
:105F100053656D5F4166650054736B5F49646C65E2
:105F20000000000053656D5F4D54427566660000C9
:105F3000456C665F5363616E0000000054736B5FD5
:105F40005363616E0000000053656D5F45767446D3
:105F500069666F0053656D5F43616C69624672618B
:105F60006D657300456C665F4D74000054736B5F24
:105F70004D740000545F0000000210001801000082
:105F80001C0100006C60000000FC10000401000017
:105F90001C0100006C60000018031000EC1B0000E6
:105FA00038010000000000000000000000000000B8
:105FB00000000000000000000000000000000000E1
:105FC00000000000000000000000000000000000D1
:105FD00000000000000000000000000000000000C1
:105FE00000000000000000000000000000000000B1
:105FF00000000000000000000000000000000000A1
:106000000000000000000000000000000000000090
:106010000000000000000000000000000000000080
:106020000000000000000000000000000000000070
:106030000000000000000000000000000000000060
:106040000000000000000000000000000000000050
:106050000000000000000000000000000000000040
:106060000000000000000000000000000000000030
:106070000000000000000000000000000000000020
:106080000000000000F001204C0001200000000092
:106090000000000000000000000000000000000000
:1060A00000000000000000000000000000000000F0
:1060B00000000000000000000000000030B572B6D3
:1060C00001250D4C256000236A07012910D082F8B4
:1060D0006B3000F03F0082F86A00084805600168F4
:1060E0000029FCD105481C300360236062B630BD36
:1060F000402182F86B10ECE7401B00225C0D00226F
:10610000FCB54FF00052D02082F8C3002B4F386806
:1061100048B140F29B70D0844520A2F85200A2F80A
:106120005200FA2008E040F22F30D0843120A2F84B
:106130005200A2F85200BC20402482F8204044259E
:1061400082F8205000234FF49676CDE9006319467B
:1061500005E00099491E00910199491C0191814275
:10616000F7D30FE082F8204082F82050CDE9006399
:10617000194605E00099491E00910199491C0191B9
:106180008142F7D392F82010C906EBD482F8C330CD
:10619000386828B141F29840D08440F2572004E09A
:1061A00041F22C00D08440F2C110A2F85200A2F8B3
:1061B00052004C2082F82000FCBD0000DC040022CC
:1061C000A5FD10000100004A0705194D01FF961FAB
:1061D0000C100F23DC052C01DC052C010000000055
:1061E000D00700000000000000000309320000009A
:1061F000000000000000000000000F010A05002C54
:10620000012C01FA000000966464005E01F401C8EC
:106210000094021405F609480DD20F000000003268
:10622000200300910032000000011A0503021A0445
:1062300001013F0244000003000100800000000053
:106240001E01400696000800E50064001F040000DF
:1062500010000001980A0B6400000000000000001C
:1062600003001005101400000000000000000000F2
:106270000000024B03320064283C401F401F32A044
:106280000FB80BA00FB80B2D0D64640000000000C8
:10629000003C000045960000050C000003010000D2
:1062A000060900004080004080000000000000005F
:1062B00000000000000000000000000000000000DE
:1062C00000000000000000000000000000000000CE
:1062D00000000000ECECECECECEC00000000000036
:1062E000000000002D2D2D2D2D2D00003C3C3C3CB0
:1062F0003C3C000023232323232300000A010F1921
:106300000F1400000000000000000000000000006A
:10631000000000000000000000000000000000007D
:10632000000000000000000000000000000000006D
:10633000000000000000000000000000000000005D
:10634000000000000000000000000000000000004D
:1069A000000002000000000000000000FD100000D8
:1069B000000000000000000000000000EF7639C673
:0469C0007DC323452B
:00000001FF
